:040000008031D6284D
:10000800803120007F08F3000B1D6F2800000000DE
:100018008530200095000B11F01E701A15288D12DE
:100028002A28F01A701E21280D128D1E1C280D1664
:1000380020008D160D1A8D122B28F01E2628103040
:100048008D068D12701E2B2820308D060D12033060
:1000580021004B02F43003194A02031843280130E7
:10006800CA070030CB3D03304B06031D3D28F33053
:100078004A06031D5B28B430200095005B28210048
:10008800CA01CB017014701F51280130A00700303D
:10009800A13D0030A23D0030A33D50080319562869
:1000A8000130D002510803195B280130D102CA304F
:1000B80021005702031865280130F2007208D7079B
:1000C8006F28D701F014F11C6B282030F006711C42
:1000D8006F281030F0068B188B102000911ECA284C
:1000E80023001908F2007208F40020009112F01998
:1000F800CA28FA08031D85280230F2007208210078
:10010800CE007408F2007A08203E8600023087008C
:10011800720881007A08013A0319A028B1283330FF
:100128009B2898280A309B2804309B280230F2002C
:1001380072082100CE00B1287408453A031998289E
:100148000C3A03199828203A031996281C3A0319DF
:100158009528023A031993289A280130F200720868
:10016800FA077A08353A031DBC28FA012100CE01A6
:1001780074082A3A031DC5287A0821004E02031C78
:10018800F01523009D1CCA281D121D162000121AE6
:100198001212111B111391199111921992117308CE
:1001A800FF0009008031D828F001F101FA01A030E0
:1001B80084000030850048308731FA2780312030AC
:1001C8008400013085004D308731FA278031A03016
:1001D80084000130850040308731FA278031203093
:1001E80084000230850035308731FA2720008331BA
:1001F800C72BF01C5C2AF0108C3198248031003019
:100208008D319625803105302100520203181029BE
:1002180005304F02031C16299D31A42580319D31DC
:100228007925803186311A26803121004108200045
:10023800AE00210042082000AF0021004308200042
:10024800B00021002C082000AB0021002D08200060
:10025800AC0021002E082000AD0097314C278031DA
:1002680020002B08BE002C08BF002D08C00000305D
:10027800BB007A30BC004430BD009631A3268031E3
:1002880020003B08CB003C08CC003D08CD00943151
:10029800F224803120004E082200DC0020004D08A6
:1002A8002200DB0020004C082200DA0020004B0866
:1002B8002200D90000302000BB007A30BC00443056
:1002C800BD000830513E860001308700403FA30042
:1002D800413FA400423FA500433FA6009F3132277B
:1002E800803120002308BE002408BF002508C00074
:1002F8009631A326803120003B082100B800200059
:100308003C082100B90020003D082100BA00220065
:1003180056082302031D922955082202031C9B2913
:1003280001302000E60066082100D6079D2921003B
:10033800D60100302000CB008230CC004230CD0006
:1003480021003E082000CE0021003F082000CF00F9
:10035800210040082000D0009F31C42780310318B5
:10036800BC2901302000E60066082100D507BE2917
:100378002100D501701F1F2A22002E089E31082651
:10038800803120002308CB002408CC002508CD00AC
:10039800210038082000CE00210039082000CF00B5
:1003A80021003A082000D0009F31C427803103186B
:1003B800E42901302000E60066082100D407E62978
:1003C8002100D40100302000CB00C830CC004230DE
:1003D800CD00210041082000CE0021004208200065
:1003E800CF00210043082000D0009F31C42780316E
:1003F80003180E2A22002C08023A031D062A883107
:10040800F020803122002C08033A031D0E2A8A317D
:10041800B922803120008D19552A3030F500753009
:10042800F6009D319725803120008D19552A90318D
:1004380035208031552A210053089E310826803105
:1004480020002308CB002408CC002508CD0021007B
:1004580038082000CE00210039082000CF002100F4
:100468003A082000D0009F31C42780310318432A5E
:1004780001302000E60066082100D407452A210043
:10048800D40120000D19552A3030F5007530F600DA
:100498009D319725803120000D19552A94316C24FF
:1004A80080319131C821803100308931D2218031A9
:1004B800701C08007010A03021009E0001309D00C3
:1004C8000230F5000030F6009D319725803121007B
:1004D8009D149D186D2A1C082000E600E701660897
:1004E8002100E800200067082100E9000830E8350D
:1004F800E90D890B7B2A1B082000E600E701660846
:100508002100E807200067082100E93D00302000AD
:10051800AB00A030AC003B30AD00210069082000E2
:10052800A401A407210068082000A301A3079D31A6
:10053800C625803120002308AE002408AF00250816
:10054800B00097314C27803120002B082100EA00A9
:1005580020002C082100EB0020002D082100EC00D1
:100568006A082000AB0021006B082000AC002100C5
:100578006C082000AD0021006A082000AE002100B0
:100588006B082000AF0021006C082000B0009731F4
:100598004C27803120002B082100BE0020002C08A9
:1005A8002100BF0020002D082100C000C930200014
:1005B800AB007230AC004130AD0021003E08200095
:1005C800AE0021003F082000AF00210040082000B5
:1005D800B00097314C27803120002B082100BE0045
:1005E80020002C082100BF0020002D082100C00099
:1005F8003E082000BE0021003F082000BF00210067
:1006080040082000C00021006A082000AE00210038
:100618006B082000AF0021006C082000B000B33048
:10062800AB00A930AC004230AD0097314C27803187
:1006380020002B08BB002C08BC002D08BD009D31F4
:100648008E25803120003B08C1003C08C2003D08CF
:10065800C3008B31A223803120003E082100BE0058
:1006680020003F082100BF00200040082100C000F2
:100678001F302000BE000C30BF004330C0002100F6
:100688003E082000C10021003F082000C2002100D0
:1006980040082000C3008B31A223803120003E088F
:1006A8002100BE0020003F082100BF0020004008B4
:1006B8002100C000701F080024082000E600210067
:1006C80025082000E700210026082000E800210076
:1006D80027082000E90021002C082000CB00210079
:1006E8002D082000CC0021002E082000CD009431D8
:1006F800F224803120004B08EA004C08EB0000305F
:10070800EB1BFF30EC00ED006A08E6076B08E73DDD
:100718006C08E83D6D08E93D69082100A700200044
:1007280068082100A600200067082100A500200015
:1007380066082100A400220059082100280720008B
:10074800E60022005A082100293D2000E700220087
:100758005B0821002A3D2000E80022005C082100F7
:100768002B3D2000E90069082100AB002000680843
:100778002100AA00200067082100A90020006608BF
:100788002100A800080095317925833137309D3143
:10079800F0258331003A0319F42BF50137309E31E7
:1007A800BD2683311030F5002730F6009D3197259E
:1007B80083319031002083319E313F2683311030C0
:1007C800F5002730F6009D31972583319231F222CA
:1007D80083311030F5002730F6009D31972583319D
:1007E80093316C23833190310020833192318B22F5
:1007F800833100302100B5000030B6000030B7006A
:100808000030BB000030BC000030BD000030A70045
:100818000030A6000030A5000030A4000030AB0076
:100828000030AA000030A9000030A8006400701C45
:100838001B2C70106400701C1F2C7010F0127016A6
:10084800F110711000302100A3000030A200003028
:10085800A1000030A0008030C4000030C500C601EF
:10086800C7016400F01D3B2C8E31B52683318031E1
:10087800FD208331701FF22D22002C08043A031D3D
:10088800DD2C2100D108031DDD2C22002F082300B8
:10089800E00060082100D10000302000CB00A0302B
:1008A800CC004030CD000030BB007A30BC00443072
:1008B800BD00220025082000A401A4072200240866
:1008C8002000A301A3079D31C625833120002308FA
:1008D800BE002408BF002508C0009631A326833136
:1008E80020003B08CE003C08CF003D08D0009F31D7
:1008F800C4278331031C852C00302000BE00003043
:10090800892C00302000BE008030BF003F30C0007E
:10091800210035082000C100210036082000C2004F
:10092800210037082000C3008B31A2238331200027
:100938003E082100B50020003F082100B600200035
:1009480040082100B70000302000BB007A30BC000E
:100958004430BD00220025082000A401A40722007D
:1009680024082000A301A3079D31C6258331200058
:100978002308BE002408BF002508C0009631A3261E
:10098800833120003B08CB003C08CC003D08CD005B
:10099800210035082000CE00210036082000CF00B5
:1009A800210037082000D0009F31C4278331031C61
:1009B800F0172100D008031D2D2DFF304502FC3013
:1009C8000319440203182D2D7016A0302000A00032
:1009D8000130A1005530A2000130A3000430A4006A
:1009E8000030A5009F315C27833121004508200095
:1009F800A201A207210044082000A101A107043098
:100A08002300E00060082000A3009E31E026833127
:100A180004302100C4070030C53D0130C60700304E
:100A2800C73D22002C08043A031D1E2D2100D001C9
:100A3800D00A252D22002F082300E000600821009D
:100A4800D000D030F5000730F6009D31972583316E
:100A580070121030203E8600013087001600010415
:100A68000319572D220030082300E0002200310826
:100A78002300E100E201E301630821002302031DD2
:100A8800552D2300620821002202031D552D230045
:100A9800610821002102031D552D23006008210053
:100AA80020020318F0170430210055020318602DA6
:100AB80004305402031C622DF017701507305202DF
:100AC80003186A2D07304F02031C6C2DF0177015A0
:100AD800043056020318722DF01F352CA030200068
:100AE800A0000130A1005530A2000130A30004305D
:100AF800A4000030A5009F315C2783312100450800
:100B08002000A201A207210044082000A101A1079A
:100B180004302300E00060082000A3009E31E02696
:100B28008331FF3021004502FC30031944020318C9
:100B3800A52D0430C4070030C53D0130C60700307C
:100B4800C73D8830F5001330F6009D319725833175
:100B5800FF302300E0006008A000FF30E0006008DC
:100B6800A100FF30E0006008A200FF30E00060084C
:100B7800A300210045082000A201A2072100440883
:100B88002000A101A10704302300E0006008200034
:100B9800A3009E31E026833101302100C6070030D2
:100BA800C73D7013F013F0127016701DDD2DF1148F
:100BB80071140030B5000030B6000030B7000030C6
:100BC800BB000030BC000030BD000030A300003086
:100BD800A2000030A1000030A000352C0430210014
:100BE80055020318FB2D04305402031C062E003056
:100BF800B5000030B6000030B7007015F01270165E
:100C0800F11471140730520203180E2E07304F02E8
:100C1800031C352C0030B5000030B6000030B7009A
:100C28007015F0127016F1147114352C2100370864
:100C380036043504031D2A2E00302000DE00003063
:100C4800DF000030E0009331E6230800210041086E
:100C58002000CB00210042082000CC0021004308DE
:100C68002000CD000030CE00C830CF004230D00088
:100C78009F31C4278631031C080000302000BB00C8
:100C88007A30BC004430BD0021002C082000BE0092
:100C980021002D082000BF0021002E082000C000E0
:100CA8009631A326863120003B08E3003C08E40087
:100CB8003D08E5006308CB006408CC006508CD005A
:100CC800D730BE00A330BF00BB30C00021003508BC
:100CD8002000C100210036082000C200210037088A
:100CE8002000C3008B31A223863120003E08CE00AD
:100CF8003F08CF004008D0009F31C4278631031831
:100D0800C52ED7302000CB00A330CC003C30CD001E
:100D1800210035082000BE00210036082000BF0051
:100D2800210037082000C0006308BB006408BC002D
:100D38006508BD009D318E25863120003B08C10025
:100D48003C08C2003D08C3008B31A2238631200035
:100D58003E08CE003F08CF004008D0009F31C4278E
:100D680086310318BE2ED7302000BE002330BF00C6
:100D78003C302C2FD7302000BE002330BF003B3042
:100D88002C2FD7302000BE00A330BF003B30C0005E
:100D9800210035082000C100210036082000C200CB
:100DA800210037082000C3008B31A22386312000A0
:100DB8003E08CB003F08CC004008CD006308CE00B9
:100DC8006408CF006508D0009F31C4278631031816
:100DD800482F20006308BE006408BF006508C000F3
:100DE800210035082000BB00210036082000BC0087
:100DF800210037082000BD009D318E258631200056
:100E08003B08C1003C08C2003D08C3008B31A22347
:100E1800863120003E08CB003F08CC004008CD00BA
:100E2800D730CE00A330CF003C30D0009F31C4274C
:100E380086310318262FD7302000BE002330BF008C
:100E4800BC302C2FD7302000BE002330BF00BB3071
:100E5800C00021002F082000C10021003008200018
:100E6800C200210031082000C3008B31A223863143
:100E780020003E082100AF0020003F082100B000FC
:100E8800200040082100B10021002F082000CB00DD
:100E9800210030082000CC00210031082000CD00BE
:100EA8000030CE000030CF00BF30D0009F31C427C3
:100EB80086310318662F00302100AF000030B000E3
:100EC800BF30B10000302000CB000030CC003F30F4
:100ED800CD0021002F082000CE002100300820007E
:100EE800CF00210031082000D0009F31C42786316F
:100EF8000318852F00302100AF000030B0003F30CC
:100F0800B1002100310830042F04031908002F080C
:100F18002000BE00210030082000BF002100310859
:100F28002000C000210035082000C100210036083B
:100F38002000C200210037082000C3008B31A22303
:100F4800863120003E08DE003F08DF004008E00050
:100F58009331E623080080302100C4000030C5002A
:100F680045082000A401A407210044082000A3018B
:100F7800A3070430A8002808A5009F318A278731D5
:100F880004302100C4070030C53D2000A901A90A8A
:100F9800AA0104302A020318EC2F2A08A03E860072
:100FA8000130870001089D317E25873120002A08FD
:100FB800A03E8600013087000108FF3A031DA90101
:100FC8000130A8002808AA0704302A02031CD12FE0
:100FD80064002000A908031D0800FF302100450215
:100FE800FB300319440203180800B42F6400800181
:080FF8000131890BFB2F0034CD
:10100200F70131307702031808007708203E860086
:101012000230870001089D317E2588310130F600BB
:101022007608F707022802309F31092788317608AF
:101032002000D201D2077508D101D10704309F31B7
:101042000927883176082000D001D0077508CF0122
:10105200CF0722006B082000CF0222006C0820007C
:10106200D03B06309F310927883176082000D40111
:10107200D4077508D301D30708309F310927883177
:1010820076082000D601D6077508D501D5072200BB
:101092006B082000D50222006C082000D63B5208C3
:1010A2005104031D612891302100DE00AD30DF00C4
:1010B2003E30E0000030E1002030E2004230EC2817
:1010C20020004F09CB005009CC00CB0A0319CC0AEF
:1010D20055084B07A30056084C3DA4009D31C62578
:1010E200883120002308BB002408BC002508BD006D
:1010F2005109CD005209CE00CD0A0319CE0A530878
:101102004D07A30054084E3DA4009D31C6258831E9
:1011120020002308BE002408BF002508C000963125
:10112200A326883120003B082100DE0020003C0875
:101132002100DF0020003D082100E00020005608C9
:10114200A401A4075508A301A3079D31C625883130
:1011520020002308AE002408AF002508B0000630A6
:10116200D83E86008701403FAB00413FAC00423F82
:10117200AD0097314C27883120002B08BB002C088A
:10118200BC002D08BD009D318E25883120003B0812
:10119200BE003C08BF003D08C0005408A401A407DB
:1011A2005308A301A3079D31C625883120002308D7
:1011B200C1002408C2002508C3008B31A223883154
:1011C20020003E082100E10020003F082100E2004B
:1011D200200040082100E3009E3123260800210060
:1011E2003D083C043B040319080000302000BB000A
:1011F2007A30BC004430BD00210041082000BE000E
:10120200210042082000BF00210043082000C00046
:101212009631A326883120003B08E3003C08E40015
:101222003D08E5006308BB006408BC006508BD001A
:1012320021003B082000BE0021003C082000BF0026
:1012420021003D082000C0009631A32688312000ED
:101252003B082100B20020003C082100B30020001E
:101262003D082100B40000302000BB007A30BC00F1
:101272004430BD00220029082000A401A407220056
:1012820028082000A301A3079D31C625883120002C
:101292002308BE002408BF002508C0009631A326FB
:1012A200883120003B08CB003C08CC003D08CD0033
:1012B200210032082000CE00210033082000CF0098
:1012C200210034082000D0009F31C4278831031840
:1012D200972900302000BB007A30BC004430BD00AA
:1012E200220029082000A401A407220028082000C7
:1012F200A301A3079D31C625883120002308BE0023
:101302002408BF002508C0009631A326883120009A
:101312003B082100B20020003C082100B30020005D
:101322003D082100B400F012F1149B29F11C9B2905
:10133200F110F016210037083406031DA6293608DD
:101342003306031DA62935083206031908003208A0
:10135200B5003308B6003408B7002F082000BE00DD
:10136200210030082000BF00210031082000C00009
:10137200210035082000C100210036082000C200EB
:10138200210037082000C3008B31A22388312000BE
:101392003E08DE003F08DF004008E0009331E6230C
:1013A20008002000DA00210023082200D4002100D6
:1013B20022082200D300210021082200D2002100AD
:1013C20020082200D100210041082000CB0021008A
:1013D20042082000CC00210043082000CD009431B7
:1013E200F224893120004C082200D601D6072000C1
:1013F2004B082200D501D50721002C082000CB0084
:1014020021002D082000CC0021002E082000CD0054
:101412009431F224893120004C082200D801D807E7
:1014220020004B082200D701D70700302000A3007C
:101432000030A2000E30A1001030A00021002708C9
:101442002000A700210026082000A6002100250870
:101452002000A500210024082000A4009031C22011
:101462008931200023082200E00020002208220007
:10147200DF00200021082200DE00200020082200D8
:10148200DD0000302000A3000030A2000E30A100D9
:101492001030A00021002B082000A70021002A08FC
:1014A2002000A600210029082000A500210028080C
:1014B2002000A4009031C22089312000230822009C
:1014C200E400200022082200E3002000210822007C
:1014D200E200200020082200E10021003E08200056
:1014E200CB0021003F082000CC0021004008200052
:1014F200CD009431F224893120004C082200E6010B
:10150200E60720004B082200E501E50758085704CA
:10151200031D912A6C08EA01EA076B08E901E90751
:1015220020005A0803190800A030A0000130A100D1
:101532005130A2000130A3001C30A4000030A500ED
:101542009F315C2789312000DB011C305B020318CC
:1015520008005B08A03E86000130870001089D312B
:101562007E25893101302000D9005908DB07A62ADF
:101572002200270826040319080000302000BB00BF
:101582007A30BC004430BD00210041082000BE007A
:10159200210042082000BF00210043082000C000B3
:1015A2009631A3268A3120003B08E3003C08E40080
:1015B2003D08E500220027082000A401A40722001C
:1015C20026082000A301A3079D31C6258A312000E9
:1015D2002308BB002408BC002508BD006308BE0028
:1015E2006408BF006508C0009631A3268A31200036
:1015F2003B082100B20020003C082100B30020007B
:101602003D082100B40000302000BB007A30BC004D
:101612004430BD00220029082000A401A4072200B2
:1016220028082000A301A3079D31C6258A31200086
:101632002308BE002408BF002508C0009631A32657
:101642008A3120003B08CB003C08CC003D08CD008D
:10165200210032082000CE00210033082000CF00F4
:10166200210034082000D0009F31C4278A3103189A
:10167200672B00302000BB007A30BC004430BD0034
:10168200220029082000A401A40722002808200023
:10169200A301A3079D31C6258A3120002308BE007D
:1016A2002408BF002508C0009631A3268A312000F5
:1016B2003B082100B20020003C082100B3002000BA
:1016C2003D082100B400F012F1146B2BF11C6B2BBE
:1016D200F110F016210037083406031D762B360868
:1016E2003306031D762B350832060319080032082B
:1016F200B5003308B6003408B7002F082000BE003A
:10170200210030082000BF00210031082000C00065
:10171200210035082000C100210036082000C20047
:10172200210037082000C3008B31A2238A31200018
:101732003E08DE003F08DF004008E0009331E62368
:10174200080020003E08C4003F08C5004008C6004B
:101752000310450D460DC7004708CA004108C400E2
:101762004208C5004308C6000310450D460DC700D8
:101772004708C9004A080319CA2B49084A02031834
:10178200D12B4A03FF3A4907C40019304402031C13
:10179200D12B4108BE004208BF004308C000080028
:1017A2004908031908004A0849020318E02B4903B3
:1017B200FF3A4A07C40019304402031808000630F1
:1017C200C4004408C800C01BC817C31B4817BF1772
:1017D200FF30BE05FF30BF050030C005C217FF3025
:1017E200C105FF30C2050030C30549084A0203188B
:1017F2001C2C0130C135C20DC30D890BFB2B0130EE
:10180200C90249084A060319172C0130C8024808C0
:1018120007390319172CFA2B0130C036BF0CBE0C46
:10182200890B0E2C0130C4004408CA074A08490635
:101832000319412C0D2C4A0849020318412C01308E
:10184200BE35BF0DC00D890B212C0130CA024908DB
:101852004A0603193D2C0130C8024808073903190A
:101862003D2C202C0130C336C20CC10C890B342C08
:101872000130C4004408C9074A084906031D332C35
:10188200C81F532CFF30BE06FF30BF06FF30C00614
:101892000130BE07003003180130BF0700300318C3
:1018A2000130C007481F652CFF30C106FF30C20659
:1018B200FF30C3060130C107003003180130C207F0
:1018C200003003180130C307C8013E08C1073F08B2
:1018D200C23D4008C33DC31F802CFF30C106FF300C
:1018E200C206FF30C3060130C107003003180130C1
:1018F200C207003003180130C307C801C80A4108F3
:10190200F5004208F6004308F7004A08C4004408FC
:10191200F8004808C5004508F900923128227508E8
:101922002000BE007608BF007708C00008009D3185
:1019320074258C31D0309D3185258C3118309D3104
:1019420085258C319D3179258C312000D8012000EC
:101952005808183A0319D02C9D3174258C31D13096
:101962009D3185258C3101309E315B268C312000E2
:10197200D4005408DA0001309E315B268C312000FD
:10198200D4005408D90000309E315B268C312000EF
:10199200D4005408D8009D3179258C31A82C5A08DE
:1019A200FF3A031DDE2C5908FF3A031DDE2C0130DD
:1019B200D40054082100D20708002100D2012000DF
:1019C200DA1FE72C2200E701E801FA2C200059086F
:1019D200D400D5015A08D600D7015608D700D6013F
:1019E200540856072200E70020005508573D220000
:1019F200E8000330D83E86008701403F2000BE0049
:101A0200413FBF00423FC000210058082000AB0008
:101A1200210059082000AC0021005A082000AD0026
:101A2200220068082000A401A40722006708200001
:101A3200A301A3079D31C6258C3120002308AE00E7
:101A42002408AF002508B00097314C278C312000C4
:101A52002B08C1002C08C2002D08C3008B31A22321
:101A62008C3120003E082100C10020003F082100E7
:101A7200C200200040082100C30041082000BE002F
:101A8200210042082000BF00210043082000C000BE
:101A920021002C082000AB0021002D082000AC0002
:101AA20021002E082000AD000C30D83E86008701B0
:101AB200403FAE00413FAF00423FB00097314C275C
:101AC2008C3120002B08C1002C08C2002D08C30055
:101AD2008B31A2238C3120003E082100C10020005E
:101AE2003F082100C200200040082100C300410835
:101AF2002000CB00210042082000CC002100430836
:101B02002000CD000030CE000030CF000030D000E9
:101B12009F31C4278C310318080000302100C10016
:101B22000030C2000030C30008002000D900D908EC
:101B3200031DA82D2100370836043504031DA82DE6
:101B42000030AC000030AD000030AE0008009D3126
:101B520074258D31D0309D3185258D3138309D31C0
:101B620085258D319D3179258D312000D8012000C8
:101B72005808383A0319E02D9D3174258D31D13042
:101B82009D3185258D3101309E315B268D312000BE
:101B9200D4005408DB0001309E315B268D312000D9
:101BA200D4005408DA0000309E315B268D312000CB
:101BB200D4005408D8009D3179258D31B82D5B08A9
:101BC200FF3A031DEE2D5A08FF3A031DEE2D013098
:101BD200D40054082100CF0708002100CF012000C3
:101BE200DB1FFE2D2200E901EA0100302100AC00DA
:101BF2000030AD000030AE00080020005A08D400CA
:101C0200D5015B08D600D7015608D700D601540883
:101C120056072200E90020005508573D2200EA003D
:101C22002000590803191D2E22006A08EC01EC0756
:101C32006908EB01EB07200022006C082000A401D8
:101C4200A40722006B082000A301A3079D31C6252B
:101C52008D3120002308BB002408BC002508BD00EC
:101C62009D318E258D3120003B08BE003C08BF000F
:101C72003D08C00022006A082000A401A407220037
:101C820069082000A301A3079D31C6258D312000DC
:101C92002308C1002408C2002508C3008B31A223F7
:101CA2008D3120003E082100AC0020003F082100B9
:101CB200AD00200040082100AE002C082000CB001F
:101CC20021002D082000CC0021002E082000CD008C
:101CD2000030CE000030CF000030D0009F31C4274A
:101CE2008D3103187B2E00302100AC000030AD0096
:101CF2000030AE000930D83E86008701403F200008
:101D0200BE00413FBF00423FC00021002C0820001E
:101D1200AB0021002D082000AC0021002E0820007D
:101D2200AD000630D83E86008701403FAE00413FFD
:101D3200AF00423FB00097314C278D3120002B0875
:101D4200C1002C08C2002D08C3008B31A223200041
:101D52003E082100AC0020003F082100AD00200019
:101D620040082100AE00080024002008243A03198C
:101D7200C72FFD2F701BFD2F94316C248E31FD2F48
:101D8200701FFD2F903135208E31FD2F701BFD2FDE
:101D9200210047084604031DD12E90317B208E314D
:101DA200210046089D317E258E31210047089D3154
:101DB2007E258E3122002C08043A031DE22E0130CA
:101DC200E42E22002F089D317E258E318731AF27E8
:101DD2008E31FD2F701BFD2F913115218E31FD2F7C
:101DE200701BFD2F883114208E31FD2F701BFD2FAB
:101DF20096310A268E31FD2F903100208E319E3190
:101E02003F268E311030F5002730F6009D319725A0
:101E12008E319231F2228E31FD2F20302000A0002F
:101E22000230A1002030A2000130A3003130A40012
:101E32000030A5009F315C278E31883101208E3120
:101E4200FD2F20302000A0000130A1002230A2008E
:101E52000230A3003130A4000030A5009F315C277E
:101E62008E319E313F268E311030F5002730F6003C
:101E72009D3197258E3192318B228E31FD2F01308B
:101E82008931D2218E31FD2F14309D317E258E3144
:101E9200FD2F9D31B3258E31FD2F701BFD2F02309A
:101EA2009F3109278E3176082100CD01CD077508B3
:101EB200CC01CC0700302000BB007A30BC0044309B
:101EC200BD0021004D082000A401A40721004C08F8
:101ED2002000A301A3079D31C6258E3120002308CF
:101EE200BE002408BF002508C0009631A3268E310B
:101EF20020003B082100B50020003C082100B6006C
:101F020020003D082100B70035082000DE00210036
:101F120036082000DF00210037082000E00093315E
:101F2200E6238E31FD2F240022082000E300E40185
:101F32006308A3006408A400A501A50A9F318A27AB
:101F42008E31230020089D317E258E31FD2F240005
:101F520023082000E30063082300A00024002208D5
:101F62002000E300E4016308A1006408A200A301C9
:101F7200A30A9E31E0268E311030F5002730F6009C
:101F82009D3197258E31FD2F0028FD2F2400210839
:101F9200433A03194A2F063A0319A82F0C3A031998
:101FA2004E2F1B3A0319FD2E013A0319C12E053A91
:101FB2000319452F343A0319C52F063A0319C72EC0
:101FC200013A0319942F0C3A0319F12E053A031919
:101FD200F72E1E3A03190E2F013A0319BB2E073AA8
:101FE2000319FD2F013A0319EB2E033A0319402F6F
:101FF200013A0319222FFD2FF011FA010800543083
:10200200F50075082200B2006530F5007508B300CE
:102012007330F5007508B4007430F5007508B5002A
:10202200B6010730F5007508AA00AB01AB0AAC0196
:10203200AC0AC830A0000030A1008430A2000330F6
:10204200A300C830A4000030A500AD01A601A7017D
:10205200E830A8000330A900AE010530F50075088C
:10206200AF00B001B10108007013F0127016003019
:102072002100B5000030B6000030B7000030BB00D0
:102082000030BC000030BD000030A3000030A200D0
:102092000030A1000030A000FF302000A60026087A
:1020A2002300A000FF302000A60026082300A10084
:1020B200FF302000A60026082300A200FF302000E7
:1020C200A60026082300A300210045082000A20143
:1020D200A207210044082000A101A1070430A600A4
:1020E2002608A3009E31E02601302100C6070030F9
:1020F200C73D080080302100C4000030C500C60181
:10210200C70145082000A401A407210044082000BB
:10211200A301A3070430A8002808A5009F318A273D
:10212200903104302100C4070030C53D0130C6079C
:102132000030C73D2000A901A90AAA0104302A02E1
:102142000318B4282A08A03E86000130870001083F
:10215200FF3A031DA9010130A8002808AA0704308C
:102162002A02031CA32864002000A908031D0800FA
:10217200FF3021004502FB30031944020318080016
:10218200822800302000AB000030AA000030A900F5
:102192000030A800230822042104200403190C297A
:1021A200AC01AC0AA31BE1280130A035A10DA20DA0
:1021B200A30D890BD6280130F5007508AC07D3288A
:1021C2000130A835A90DAA0DAB0D890BE228230811
:1021D2002702031DF62822082602031DF6282108DD
:1021E2002502031DF62820082402031C01292008C9
:1021F200A4022108A53B2208A63B2308A73B2814DA
:102202000130A336A20CA10CA00C890B02290130CB
:10221200AC02031DE1282B08A3002A08A20029080A
:10222200A1002808A000080002309F31092791313F
:1022320076082100CD01CD077508CC01CC074D08E9
:102242004C04031D2A294530D8008030D9003F3084
:102252006029220068082000A401A4072200670860
:102262002000A301A3079D31C62591312000230838
:10227200BB002408BC002508BD0021004D08200039
:10228200A401A40721004C082000A301A3079D314B
:10229200C625913120002308BE002408BF0025086E
:1022A200C0009631A326913120003B082100D800BE
:1022B20020003C082100D90020003D082100DA005E
:1022C2000030DB000030DC000030DD009E312326D0
:1022D20008002000DD00BE295A08DC005908DB0096
:1022E2005C0DDC0CDB0C5C0DDC0CDB0C5B082500F4
:1022F200910020005A08DC005908DB005C0DDC0C60
:10230200DB0C5B1C87292500931689292500931273
:102312002000591C8F29250013169129250013121C
:1023220021000E118E14080020005A08DC00590802
:10233200DB005C0DDC0CDB0C5C0DDC0CDB0C5B08ED
:102342002500980020005A08DC005908DB005C0DCB
:10235200DC0CDB0C5B1CB02925009A16B229250087
:102362009A122000591CB82925001A16BA292500EC
:102372001A1221000E158E10080020005D08013A85
:1023820003196D29033A03199529C729080000305A
:102392002000CB002030CC004230CD0021003E088E
:1023A2002000CE0021003F082000CF00210040087D
:1023B2002000D0009F31C42791310318E429FF3057
:1023C200260098000800210038082000CB002100D8
:1023D20039082000CC0021003A082000CD009431B9
:1023E200F224913120004C08DA004B08D900D9358B
:1023F200DA0DD935DA0D5908203EDB0000305A3D9E
:10240200DC005C08803AFF0080307F02031D0B2A4B
:1024120040305B020318122A40302000DB000030FB
:10242200DC0020005C08803AFF0081307F02031D3F
:102432001C2A00305B02031C232AFF302000DB0031
:102442000030DC0020005B082600980008007808B5
:102452000319302A770876047504031D422A0030D6
:10246200F5000030F6000030F700080001302000CF
:10247200A0002008F8070130F736F60CF50C890B9E
:102482003D2AFE30770503195C2A372A01302000E5
:10249200A0002008F8070130F507003003180130CA
:1024A200F607003003180130F7070130F736F60C53
:1024B200F50C890B572AFF3077050319692A472A39
:1024C2000130F8020130F535F60DF70D890B642A5B
:1024D200F61F612A7818732AFF30F5057F30F6055A
:1024E200FF30F7050310F80C78082000A000A101C6
:1024F200A2011030A035A10DA20D890B7B2A200864
:10250200F5042108F6042208F704790803190800E3
:10251200F717080000302000A3000030A40031307B
:10252200A8002808A5009F318A2792312030200078
:10253200A0000130A100A030A2000130A300313080
:10254200A4000030A5009F315C2792310B3022009D
:102552002F02031CB22A05302000A80028082200FE
:10256200AF002D08210053020318BD2A5308200092
:10257200A80028082200AD002200AE08031DC82AC8
:10258200210053082000A80028082200AE002508D8
:1025920021004902031DD12A2200240821004802F9
:1025A2000318DC2A49082200A501A50721004808D2
:1025B2002200A401A4072200290821004902031DC8
:1025C200E62A2200280821004802031808004908C8
:1025D2002200A901A907210048082200A801A80792
:1025E200080045302100D8008030D9003F30DA00A1
:1025F2000030DB000030DC000030DD009130DE0016
:10260200AD30DF003E30E0000030E1002030E2007B
:102612004230E300D730E400A330E5003C30E6006E
:10262200BE302000A60026082100E700A0302000CE
:10263200A0000130A100D830A2000030A300103069
:10264200A4000030A5009F315C2792316430200045
:10265200A1000030A2001030A6002608A3009E317F
:10266200E02692311030F5002730F6009D31972593
:10267200923110302100C8002730C9000A302000F2
:10268200A60026082300A0007E302000A100003012
:10269200A200A301A30A9E31E02692311030F50078
:1026A2002730F6009D319725923164302000A60034
:1026B20026082100D30064302000A600260823004B
:1026C200A0007F302000A1000030A200A301A30AD5
:1026D2009E31E026080064302000A3000030A400F0
:1026E2001030A8002808A5009F318A279331D830DE
:1026F2002000A0000030A100A030A2000130A30001
:102702001030A4000030A5009F315C2793312100D6
:102712005D085C045B040319912B9231F222933120
:102722007E302000A3000030A400A501A50A9F313D
:102732008A279331230020082000A800A901280835
:102742002100C800200029082100C9004908F6011B
:10275200F6074808F501F507E830F7000330F800FE
:102762009E317B26933176082100C901C90775087D
:10277200C801C807490848040319C62B3A30490260
:10278200993003194802031CCA2B1030C8002730A5
:10279200C9007F302000A3000030A400A501A50AD3
:1027A2009F318A279331230020082000A80028089F
:1027B2002100D30097305302031C0800643020002C
:1027C200A80028082100D300080020005E08CB00E2
:1027D2005F08CC006008CD000030CE000030CF0092
:1027E2000030D0009F31C42793310318FF2B0030F3
:1027F2002000DE000030DF000030E00020005E0834
:10280200CB005F08CC006008CD000030CE008030E5
:10281200CF004030D0009F31C427933103183B2CA6
:10282200210067089E310826933120002308AE005C
:102832002408AF002508B0005E08AB005F08AC00BA
:102842006008AD0097314C27933120002B08CB0054
:102852002C08CC002D08CD009431F22493312000B5
:102862004C08DA01DA074B08D901D9070230913155
:102872006A210800210067362000E100E2016108B8
:10288200A3006208A4009E319B26933120002308F6
:10289200AE002408AF002508B0005E08AB005F0858
:1028A200AC006008AD0097314C27933120002B0813
:1028B200CB002C08CC002D08CD009431F2249331AA
:1028C20020004C08DA01DA074B08D901D907013098
:1028D20091316A21080070117017F013F110711014
:1028E200F016701200302100A7000030A600003060
:1028F200A5000030A4000030AB000030AA00003078
:10290200A9000030A8000030A3000030A20000306F
:10291200A1000030A0008030C4000030C500C60114
:10292200C70122002F082000CB004B082100D00055
:10293200E62C00302000BB007A30BC004430BD00E1
:10294200220025082000A401A40722002408200058
:10295200A301A3079D31C625943120002308BE00A0
:102962002408BF002508C0009631A32620003B089A
:102972002100B50020003C082100B60020003D08DF
:102982002100B700080022002D089E3108262000F1
:1029920023082100BB00200024082100BC002000E5
:1029A20025082100BD00080000302100B5000030DC
:1029B200B6000030B700D001D00A22002F08200054
:1029C200CB004B082100D100080022002C08840013
:1029D200053004020318080098310435003E8200D5
:1029E200080020004B08CF004C08D0004D08D10051
:1029F2000310500D510DD2005208D800D808031D03
:102A02000B2D0030CE000030CD000030CC00003065
:102A1200CB0008004B08CF004C08D0004D08D10075
:102A22001730D136D00CCF0C890B122D4F08D200A3
:102A32005208D300CC17FF30CB05FF30CC05003055
:102A4200CD054B08D4004C08D5004D08D600D7015F
:102A52008E30D802D81F492D5808803A8F3E03186D
:102A62003B2D0030CE000030CD000030CC000030D5
:102A7200CB0008000130D736D60CD50CD40C890B0C
:102A82003C2D0130CF004F08D8070319622D3B2D92
:102A920018305802031C5F2D0030CE000030CD00EC
:102AA2000030CC000030CB0008000130D435D50D09
:102AB200D60DD70D890B572D0130D802D808031D2A
:102AC200562D53080319702DD409D509D609D709F3
:102AD200D40A0319D50A0319D60A0319D70A5708C3
:102AE200CE005608CD005508CC005408CB00080093
:102AF20020009E1321001D1022009113931397139F
:102B020098139A139B13013023008C008D019D139F
:102B12002F0091132100991519169916191799105A
:102B220019109913FF308C00CC308D00FF308E00CD
:102B320020008D018E01183021009700023095008F
:102B42000C3024008D0020001E1021009511151557
:102B520095101510A43023009E0090309D009F1107
:102B620008309B0001309C00E0308B0020302100B7
:102B72009100FF3020009B000C30250093000C30A8
:102B82009A000C3026009A0025009E010430200095
:102B92009C00260098019D31A42595319D3179250F
:102BA200953124001614F430F5000130F6009D3101
:102BB2009725953124001615F430F5000130F60002
:102BC2009D3197259531F0127016F1147114003071
:102BD2002000DE000030DF000030E0009331E62309
:102BE20095312000E4010A30640203180800013024
:102BF2008D31962595316030F500EA30F6009D3131
:102C020097259531640001302000E3006308E40752
:102C1200F42D00302100E4000030E5000030E60031
:102C22008C319824963102309F31092796317608EB
:102C32002100CD01CD077508CC01CC074108200049
:102C4200CB00210042082000CC00210043082000D4
:102C5200CD0021004D082000A401A40721004C084A
:102C62002000A301A3079D31C62596312000230829
:102C7200CE002408CF002508D0009F31C42796310A
:102C82000318A02E210041082000BB0021004208A9
:102C92002000BC00210043082000BD009D318E258C
:102CA200963120003B08BE003C08BF003D08C00032
:102CB20021004D082000A401A40721004C08200097
:102CC200A301A3079D31C625963120002308C10028
:102CD2002408C2002508C3008B31A22396312000AC
:102CE2003E082100E40020003F082100E50020000A
:102CF20040082100E6002C082000BB0021002D081E
:102D02002000BC0021002E082000BD000C30D83E5F
:102D120086008701403FBE00413FBF00423FC000E6
:102D22009631A326963120003B082100E4002000C2
:102D32003C082100E50020003D082100E6009E310C
:102D42002326080020003E08C1003F08C2004008B8
:102D5200C3000310420D430DC4004408C900C90852
:102D6200031DBA2E0030BB000030BC000030BD0095
:102D720008003B08C1003C08C2003D08C300031024
:102D8200420D430DC4004408CA00CA08031DD02ED8
:102D92000030BB000030BC000030BD000800003035
:102DA200C6000030C7000030C80089304A07C100A1
:102DB2004108C9023E08C1003F08C2004008C300E2
:102DC2001030C336C20CC10C890BE22E4108C4007C
:102DD2004408CA003B08C1003C08C2003D08C300C9
:102DE2001030C336C20CC10C890BF22E4108C4004C
:102DF2004408CA068030C1004108CA05BF17FF3027
:102E0200BE05FF30BF050030C005BC17FF30BB0553
:102E1200FF30BC050030BD051830C1004108C500B7
:102E22000130C635C70DC80D890B122F3D0840026F
:102E3200031D212F3C083F02031D212F3B083E02A8
:102E4200031C2A2F3B08BE023C08BF3B3D08C03B87
:102E520046140130BE35BF0DC00D890B2B2F01303A
:102E6200C502031D112F4608F5004708F600480861
:102E7200F7004908C1004108F8004A08C2004208A8
:102E8200F9009231282275082000BB007608BC00A8
:102E92007708BD00080020002B08B1002C08B20002
:102EA2002D08B3000310320D330DB4003408B50001
:102EB200B508031D632F0030AB000030AC000030BA
:102EC200AD0008002E08B1002F08B2003008B30090
:102ED2000310320D330DB4003408BA00BA08031DD2
:102EE200792F0030AB000030AC000030AD0008009C
:102EF2003A087B3EB1003108B5072B08B1002C0817
:102F0200B2002D08B3001030B336B20CB10C890BED
:102F1200852F3108B4003408BA002E08B1002F08FA
:102F2200B2003008B3001030B336B20CB10C890BCA
:102F3200952F3108B4003408BA068030B100310848
:102F4200BA05AC17AF17FF30AE05FF30AF05003042
:102F5200B0050030B6000030B7000030B8000730CE
:102F6200B1003108B9002B1CBC2F2E08B6072F0860
:102F7200B73D3008B83D0130AD36AC0CAB0C890B17
:102F8200BD2F0130AE35AF0DB00D890BC32F01300F
:102F9200B902031DB42F0930B1003108B9002B1C4E
:102FA200D82F2E08B6072F08B73D3008B83D01309C
:102FB200AD36AC0CAB0C890BD92F0130B836B70C3F
:102FC200B60C890BDF2F0130B902031DD02F360852
:102FD200F5003708F6003808F7003508B100310867
:102FE200F8003A08B2003208F90092312822750836
:102FF2002000AB007608AC007708AD0008009431E1
:10300200F12C94319A2C9431C42C9431F12C9431BA
:02301200D52CBB
:103AE8009D31DB252400161408009D31DB252400B8
:103AF80016150800F50023009E1C7F2D75089A00F6
:103B080008002000A0009D31DB25200020082400AB
:103B18009100080020003D083C043B0403190800FC
:103B28008030BD0608000130F5020030F63BFF305A
:103B38007606031DA12DFF30750603190800972D81
:103B480020008E150E163830240095009601083096
:103B5800920020009111921124009417080020006F
:103B6800A001383020020318080020089D31F025F4
:103B78009D319D317E259D310130F9007908200065
:103B8800A007B52D20002308F5002408F600F7014A
:103B98008E30A6002608F800F9019231282275080F
:103BA8002000A3007608A4007708A50008000310E9
:103BB8002400141903140030093DF500F6011F30E4
:103BC8001605F70075087704F8007608F9007908F3
:103BD800780403190800DB2DF80064002300951809
:103BE800F12D7808F500F601750891007608920025
:103BF8003F30F700770895051514031015180314BE
:103C08000030093D130808002000AA002A08A60071
:103C1800A701A8012608F5002708F6002808F700DC
:103C28008E30A9002908F800F90192312822750878
:103C38002000A3007608A4007708A5000800A0309B
:103C48002000A0000130A100D830A2000030A3005D
:103C58001030A4000030A5009F315C279E316430ED
:103C68002000A1000030A2001030A6002608A30002
:103C78009E31E0260800A0302000A0000130A100FD
:103C88002030A2000130A3003130A4000030A5008C
:103C98009F315C279E3100302000A1000030A20037
:103CA8003130A6002608A3009E31E0260800200037
:103CB800A1009D31DB259E31240096159D31DB2521
:103CC8009E31240011082000A0002008A2009D3188
:103CD800DB259E31200021080319752E2400961239
:103CE800772E2400961616162000220808002000B9
:103CF800A001A101751C852E77082000A00778086F
:103D0800A13D0130F735F80D890B862E0130F636C6
:103D1800F50C890B8B2E76087504031D7E2E20006A
:103D28002108F601F6072008F501F507080020002C
:103D3800A801A41FA62EA309A409A30A0319A40A6B
:103D4800A801A80A2308F5002408F600F7018E3018
:103D5800A6002608F8002808A7002708F9009231CD
:103D6800282275082000A3007608A4007708A5007B
:103D78000800F80023009518BE2E7808F600F70111
:103D88007608910077089200750893003F30F60096
:103D980076089505200003108B1B03148B13230052
:103DA800151555309600AA30960095141511200067
:103DB800031C08008B1708009D3174259E31AE3016
:103DC8009D3185259E31200022089D3185259E3113
:103DD800200021089D3185259E312000A50123085A
:103DE80025020318062F2508A03E8600013087000B
:103DF80001089D3185259E3101302000A40024084A
:103E0800A507F32E9D31792508002000A000200881
:103E1800203E8600023087000108F700F801770885
:103E2800A1007808A2002108F800F7017708A1008E
:103E38007808A2002008013E203E86000230870054
:103E480001082107A10022080318220AA20022085B
:103E5800F601F6072108F501F50708008E30200065
:103E6800A7002708A800FF3026050319472F0130AF
:103E7800A636A50CA40CA30C890B3C2F0130A70077
:103E88002708A807372F2308F5002408F600250877
:103E9800F7002808A7002708F800F901923128221E
:103EA80075082000A3007608A4007708A50008007C
:103EB80020002308F901F9072208F801F80721086A
:103EC800F701F7072008F601F6070130A4020030D1
:103ED800A53BFF302506031D732FFF302406031969
:103EE800080078088600790887000108F500760838
:103EF800860077088700750881000130F8070030D0
:103F0800F93D0130F6070030F73D692F9D317425E2
:103F18009F31AE309D3185259F31200024089D3189
:103F280085259F31200023089D3185259F319D31AE
:103F380079259F319D3174259F31AF309D3185257D
:103F48009F312000A701250827020318BD2F013043
:103F58009E315B269F312000A6002708A03E8600E0
:103F680001308700260881000130A6002608A7072F
:103F7800A72F00309E315B269F319D31792508009F
:103F88002000CD1FDB2F4B09D1004C09D2004D0971
:103F9800D300D10A0319D20A0319D30A00305107F2
:103FA800CB000030523DCC008030533DCD00D01FB7
:103FB800F12F4E09D1004F09D2005009D300D10A80
:103FC8000319D20A0319D30A00305107CE00003072
:103FD800523DCF008030533DD0008030CD06803038
:103FE800D00650084D02031D08004F084C02031D5F
:083FF80008004E084B0208000E
:020000040001F9
:04000E001ACEDFDA4D
:10E0000041004100540069005300200041006B00B2
:10E010006B00750074006500730074006500720089
:10E020002000410053003900310037002000560025
:10E0300031002E0034002000300037002F00320065
:10E04000300031003700200043006F00700079007D
:10E0500072006900670068007400200044004C00F2
:10E060003300480052005400000000000000FF0090
:00000001FF
